S02B0000433A2F576F726B2F736F6674776172652F4F70656E424C542F5461726765742F44656D6F2F41524DEF
S1138000F40800209B810000958400009584000002
S113801095840000958400009584000095840000F8
S113802095840000958400009584000095840000E8
S1138030958400009584000095840000118500005B
S113804095840000958400009584000095840000C8
S113805095840000958400009584000095840000B8
S113806095840000958400009584000095840000A8
S11380709584000095840000958400009584000098
S11380809584000095840000958400009584000088
S11380909584000095840000958400009584000078
S11380A09584000095840000958400009584000068
S11380B09584000095840000958400009584000058
S11380C09584000095840000958400009584000048
S11380D09584000095840000958400009584000038
S11380E09584000095840000958400009584000028
S10780F0EE11AA558A
S11380F42B49072291438D462A482B492B4A00F0E9
S113810439F82B482B492C4A00F034F82B482C49D5
S11381142C4A00F02FF82C482C492D4A00F02AF858
S11381242C482D492D4A00F025F82D482D492E4A76
S113813400F020F82D482E49002200F026F82D489E
S11381442D49091A082903DB002202600430016066
S11381541E481F49884205D00268043003B490477E
S113816403BCF7E700208646EC4600200021234A9E
S11381749047FEE7884207D0521A05D003780130AD
S11381840B700131013AF9D17047884202D0027070
S11381940130FAE770471A481A490160A8E7000059
S11381A4F4080020C8BC00000000002000000020E7
S11381B40C8200000C820000B8B90000C8BC0000A6
S11381C40000002000000020B8B90000B8B9000085
S11381D4B8B90000B8B90000B8B90000B8B90000D3
S11381E4B8B90000B8B90000C5BC00000000002004
S11381F47407002074070020F4070020158400008D
S10B820408ED00E00080000019
S113820C80B500AF014B984700BF80BD3D82000094
S113821C80B500AF014B984700BF80BD8982000038
S113822C80B500AF014B984700BF80BD45AF00003F
S113823C98B500AF0A480B4B98470B48094B984725
S113824C03214FF04020094B9847094B98470146AE
S113825C60234FF461420748074CA04700BF98BD08
S113826C01000010E1AE00000100002071AB000021
S113827C81B1000000C00040C5B4000080B500AF5F
S113828C254B1B78002B15D12448254B98470346C6
S113829C012B3FD1214B1B78002B3BD0214B984712
S11382AC0246214B1A601C4B01221A701F4B0022F0
S11382BC1A702FE01D4B1B780133184A13441846CF
S11382CC174B98470346012B19D1184B1B780133D4
S11382DCDAB2164B1A70114B1A78144B1B789A425B
S11382EC18D10D4B00221A700C4B5B78FF2B11D15B
S11382FC0A4B9B78002B0DD10D4B98470AE0094B88
S113830C98470246084B1B6864339A4202D9024BC5
S113831C00221A7000BF80BD000000200400002061
S113832C41830000FD840000480000204C00002024
S113833C2D82000080B584B000AF786009480A4BE8
S113834C9847F860FB68B3F1FF3F05D0FB68DAB2DD
S113835C7B681A70012300E0002318461037BD46D1
S113836C80BD00BF00C00040D5B6000080B500AF92
S113837C0648074B984701210648074B98470022AB
S113838C01210448054B984700BF80BD2000002004
S113839CE1AE00000050024019AB0000CDAA000071
S11383AC80B582B000AF134B98477860124B1B68B2
S11383BC7A68D31AB3F5FA7F18D3104B1B78002BB9
S11383CC08D10E4B01221A70012201210C480D4BCD
S11383DC984707E0094B00221A7000220121084833
S11383EC084B9847044A7B68136000E000BF0837C9
S11383FCBD4680BDFD8400005000002054000020C8
S113840C00500240CDAA000080B500AF064B98473F
S113841C064B9847064B9847064B9847064B98478C
S113842C064B9847F8E700BF4D8400002D850000EB
S113843C0D820000AD830000358600001D82000013
S113844C80B500AF0448054B9847054B9847054B3E
S113845C984700BF80BD00BF8003C00165AF00001A
S113846C798300009D84000080B483B000AF7860F1
S113847C3960034A7B681360024A3B681360FEE769
S113848C580000205C00002080B400AFFEE700BF61
S113849C80B500AF094B98470246094BA3FB022356
S11384AC9B091846074B9847074B9847074B984727
S11384BC0020074B984700BF80BD00BF81B100006E
S11384CCD34D621049B4000011B400002DB4000067
S11384DCE184000080B483B000AF7860034A7B6809
S11384EC136000BF0C37BD4680BC70476000002091
S11384FC80B400AF024B1B681846BD4680BC704765
S113850C6000002080B400AF044B1B680133034AA5
S113851C136000BFBD4680BC704700BF60000020E4
S113852C80B582B000AF204B9847204B9847034648
S113853C03F5FA731E4A13601C4B9847034603F564
S113854C1C5310331B4A13601B4B98474FF6A963FB
S113855CBB8043F61373FB80BA88184B1A80FA88D5
S113856C164B5A804FF6FF73BB800023FB80BA88EE
S113857C134B1A80FA88124B5A804FF6A963BB80AE
S113858C40F21313FB80BA880E4B1A80FA880D4BF9
S113859C5A804EF603000C4B98470C4B984700BF7F
S11385AC0837BD4680BD00BF21B70000FD84000024
S11385BC6400002068000020898900006C00002001
S11385CC74000020700000200D8A000041B70000E8
S11385DC80B582B000AF114B1B7803F04003002B25
S11385EC17D10E4B1B7803F00203002B12D00C4B4B
S11385FC1B687B607B6804337B607B681B78FF2B78
S113860C08D17B6801331B78002B03D1054B9847A9
S113861C00E000BF0837BD4680BD00BFD006002077
S113862CC40600202D82000090B583B000AF3B4BF4
S113863C984738603B68002B2FD03B689AB2384B74
S113864C1A80384B9C894FF40060374B984703468B
S113865C9C420ED10120354B9847314B1B88002B83
S113866C1BD0334B9847334B98472D4B00221A8021
S113867C13E02C4B9C8940F606002B4B9847034681
S113868C9C420AD12C4B9847254B1B88002B04D0B9
S113869C284B9847224B00221A80284B98470246B5
S11386AC274B1B689A4225D3254B1B6803F5FA7399
S11386BC234A136000237B6019E07A6813461B017C
S11386CC9B1A5B001F4A13441F4A13600220174B6A
S11386DC9847134B1B88002B06D0154B9847154B0A
S11386EC98470F4B00221A807B6801337B607B68B0
S11386FC002BE2D0114B98470246144B1B689A424C
S113870C08D3124B1B6803F51C5310330F4A136028
S113871C0F4B984700BF0C37BD4690BDA5B8000061
S113872CCC060020800000204D9A0000BD8A000079
S113873C819D0000F5B80000699C0000FD840000D8
S113874C64000020D8060020D40600206800002015
S113875C759A000080B483B000AF78600B467B80C0
S113876C7B6803331A787B88DBB21344DAB2294B67
S113877CDA707B6802331A787B881B0A9BB2DBB2F3
S113878C1344DAB2234B9A707B685A78214B5A7093
S113879C7B681A781F4B1A701E4B9B789AB27B8895
S11387AC1B0A9BB29A420FD21A4B5B780133DAB292
S11387BC184B5A70174B5B78002B05D1154B1B7853
S11387CC0133DAB2134B1A70124BDB781A467B88DE
S11387DCDBB29A4219DA0F4B9B780133DAB20D4BA8
S11387EC9A700C4B9B78002B0FD10A4B5B7801339E
S11387FCDAB2084B5A70074B5B78002B05D1054B4A
S113880C1B780133DAB2034B1A7000BF0C37BD4628
S113881C80BC70470407002080B487B000AF0346C7
S113882C3960FB801346BB803B687B61BB88013B92
S113883C3A6813443B6118E07B691B789BB21B02BA
S113884C9AB27B6901331B789BB21344FB81FA887F
S113885CFB891344FB80FA88FB899A4202D2FB8879
S113886C0133FB807B6902337B617A693B699A42F1
S113887CE2D37A693B699A420FD17B691B789BB22C
S113888C1B02FB81FA88FB891344FB80FA88FB8961
S113889C9A4202D2FB880133FB80FB8818461C37B2
S11388ACBD4680BC704700BF80B582B000AF1422B7
S11388BC0A4900200A4B98470346FB80FB88002B8F
S11388CC05D0FB881846074B9847034601E04FF642
S11388DCFF7318460837BD4680BD00BF8E000020CC
S11388EC258800004D9A000080B584B000AF034683
S11388FCFB71184B9B789BB21B029AB2154BDB781D
S113890C9BB213449BB2143BFB81FB799AB2FB8957
S113891C1344BB811049BB89082218460F4B984756
S113892C0346BB81FA89BB890D4918460B4B984702
S113893C0346BB81BB89002B05D0BB891846094B68
S113894C9847034601E04FF6FF7318461037BD46AF
S113895C80BD00BF8E0000209A00002025880000F6
S113896CA20000204D9A000080B500AF0620024BF7
S113897C98470346184680BDF588000080B400AFC4
S113898C1B4B00221A700CE0194B1B781A46194B1E
S113899C002123F81210164B1B780133DAB2144B56
S11389AC1A70134B1B78002BEED0114B00221A704B
S11389BC11E00F4B1B7819460F4A0B461B015B1A2F
S11389CC5B001344193300221A70094B1B780133D2
S11389DCDAB2074B1A70064B1B78002BE9D0074B05
S11389EC4FF480621A8000BFBD4680BC704700BF44
S11389FC08070020F8060020D806002000070020F5
S1138A0C80B483B000AF0346FB80114B00221A7074
S1138A1C15E00F4B1B781A460E4B33F81230002B13
S1138A2C07D10B4B1B7819460A4AFB8822F81130E4
S1138A3C09E0074B1B780133DAB2054B1A70044B6F
S1138A4C1B78002BE5D00C37BD4680BC704700BFAB
S1138A5C08070020F806002080B582B000AF03465A
S1138A6CFB80104B1B680833FA88114618460E4BD2
S1138A7C98470C4B1B680D4A12781A72094B1B68E9
S1138A8C0A4A52785A72074B1B68084A92789A72AF
S1138A9C044B1B68054AD278DA7200BF0837BD460E
S1138AAC80BD00BFD40600206187000004070020AD
S1138ABC90B585B000AF0346FB71A34B1C68A34B68
S1138ACCA34A1A60A14B1B68A24A1360FB79032BBF
S1138ADC10D1637E03F00F03032B40F06887238AC5
S1138AEC002B40F064879C4B08221A709B4B9847D0
S1138AFC00F0C5BDFB79022B40F0A580984BDB78C8
S1138B0C0133DAB2964BDA70954BDB78002B19D122
S1138B1C934B9B780133DAB2914B9A70904B9B78C0
S1138B2C002B0FD18E4B5B780133DAB28C4B5A701D
S1138B3C8B4B5B78002B05D1894B1B780133DAB254
S1138B4C874B1A70874B00221A80874B00221A809D
S1138B5C637E072B02D0637E052B09D1A37E0133E0
S1138B6CDBB2A376A37E782B6BD10023637668E00B
S1138B7C637E002B00F01D87238A002B54D0A37E28
S1138B8C5A1ED2B2A276002B40F01387E37E082B38
S1138B9C08D0637E022B02D0637E012B0FD1E37EBF
S1138BAC052B0CD1002363766B4B80221A706B4B14
S1138BBC98476E4B142283F8212000F05DBEE37EAF
S1138BCC042B05D8E37E1A4603239340DBB200E062
S1138BDC3023A376E37E0133DBB2E376637E03F0CA
S1138BEC0F03013B072B00F2E48601A252F823F099
S1138BFC479100001D8C0000278C0000B7950000E5
S1138C0CBF990000B7950000BF990000B79500000C
S1138C1C564B002283F8212098E24F4B04221A7001
S1138C2C4E4B984700F06FBD637E03F00F03032B8C
S1138C3C40F0BF86484B08221A70484B984700F006
S1138C4C1EBD00F0B6BE494B1B78452B40F0B386D5
S1138C5C464B9B781B02454AD2781344414A1288EE
S1138C6C934200F3AA86414B9B789BB21B029AB2A7
S1138C7C3E4BDB789BB213449AB23A4B1A803B4B73
S1138C8C9B7903F03F03002B40F0CB86374BDB7909
S1138C9C002B40F0C686364B1A88364B1B889A42FA
S1138CAC05D1334B5A88344B1B889A420DD0334B25
S1138CBC1A882F4B1B889A4240F0B386304B1A8883
S1138CCC2B4B5B889A4240F0AC862E4B984703465C
S1138CDC1A464FF6FF739A4240F07186234B5B7A27
S1138CEC062B55D0214B5B7A012B40F06A861F4B27
S1138CFC1B7D082B40F067861C4B00221A751B4BFE
S1138D0CDB8A4FF6F672934206D9184A174BDB8A64
S1138D1C09339BB2D38205E0144A144BDB8A083323
S1138D2C9BB2D382154B184A12881A80144B174ADB
S1138D3C12881A80144B0E4A12881A80134B0C4A50
S1138D4C52881A8000F02FBED4060020C4060020DE
S1138D5CB6000020C8060020D0060020DD850000E7
S1138D6CFC060020CC060020CE0600208E0000203D
S1138D7C6C000020B8B90000BAB900009E000020B5
S1138D8CA0000020B58800009A0000209C00002060
S1138D9C00BF744B984703461A464FF6FF739A422A
S1138DAC40F01386704C18E0637E002B14D06F4B8C
S1138DBCDA8AA3889A420FD16C4B9A8AE3889A4236
S1138DCC0AD16B4B1A8823889A4205D1694B1A88AD
S1138DDC63889A4200F0DB811E34634B9C42E3D9D6
S1138DEC624B93F8213003F03F03022B1DD15F4BF0
S1138DFCDA8A614B1A80614B00221A7010E05F4BC7
S1138E0C1B781A465E4B33F812205B4B1B889A4234
S1138E1C00F08A80594B1B780133DAB2574B1A7025
S1138E2C564B1B78002BEAD000E000BF4F4B93F855
S1138E3C213003F00403002B40F0C9854B4B142262
S1138E4C83F821204F4B28221A80484B502283F858
S1138E5C2020464BDA7E494B1A70444B434AD27F4E
S1138E6CDA76424B454A1278DA77404B9A7E434B7A
S1138E7C1A703E4B3D4A927F9A763C4B3F4A12788D
S1138E8C9A773A4B5A7E3D4B1A70384B374A527F7D
S1138E9C5A76364B394A12785A77344B1A7E374BFA
S1138EAC1A70324B314A127F1A76304B334A12788D
S1138EBC1A772E4BDA7F0132D2B2DA77DB7F002BB2
S1138ECC14D12A4B9A7F0132D2B29A779B7F002B12
S1138EDC0CD1264B5A7F0132D2B25A775B7F002BCE
S1138EEC04D1224B1A7F0132D2B21A771F4B9A8AC1
S1138EFC214B1A801D4B1D4AD28A9A821B4B1E4A47
S1138F0C1288DA82204B1A4A12881A801F4B194A8B
S1138F1C12881A80164B1E4A12881A80154B1C4A4A
S1138F2C52881A8000F0F5BC00BF0024134B0022B9
S1138F3C1A705BE0114B1B7819460B4A0B461B014C
S1138F4C5B1A5B00134419331B78002B22D10B4B97
S1138F5C1B781A4613461B019B1A5B00024A9C1889
S1138F6C48E000BF75890000D80600208E00002060
S1138F7C9A0000209C0000200A070020080700200B
S1138F8CF8060020CC0600209E000020A000002043
S1138F9C6C000020894B1B781946894A0B461B012F
S1138FAC5B1A5B00134419331B78072B18D1002C64
S1138FBC0DD0824B1B781946814A0B461B015B1A58
S1138FCC5B0013441A331A78A37E9A4208D97B4B5C
S1138FDC1B781A4613461B019B1A5B00784A9C1893
S1138FEC764B1B780133DAB2744B1A70734B1B78C3
S1138FFC002B9FD0002C00F0EC84724B1C600323DC
S113900CA376A37E23760023A3750423E3750023A0
S113901CE3766D4BDB8AA3806B4B9B8AE3806B4BB3
S113902C1B8823806A4B1B88638001236376694BFE
S113903C1B782373674B5B786373664B9B78A373C2
S113904C644BDB78E373012323825F4BDB7EE37297
S113905C5D4B9B7EA3725C4B5B7E63725A4B1B7E97
S113906C237201205C4B9847574B93F8203003F044
S113907CF003502B66DD514B00221A7050E04F4B1D
S113908C1B783633554AD25C554B1A70544B1B78AB
S113909C002B54D0524B1B78012B06D1474B1B7819
S11390AC0133DAB2454B1A703AE04D4B1B78022B64
S11390BC24D1424B1B783733484AD35C042B1DD143
S11390CC3E4B1B783833454AD35C1B021AB23B4BDC
S11390DC1B7839334149CB5C1BB213431BB29AB294
S11390EC404B1A803F4B1B8840F20A62934228BFC4
S11390FC13469BB26382638AA38223E02F4B1B78B3
S113910C3733364AD35C002B1BD02C4B1B783733AC
S113911C324AD25C294B1B781344DAB2274B1A70AF
S113912C264B1B781A46284B93F820301B09DBB2CC
S113913C053B9B009A42A2DB04E000BF02E000BFA7
S113914C00E000BF204B102283F821201E4A1E4B46
S113915C93F8213043F00203DBB282F821301A4B2E
S113916C022283F82820184B042283F82920164B5A
S113917C062283F82A20144B0A2283F82B201A4B3C
S113918C2C221A80104B602283F820207BE300BF32
S113919C0C4B1C60154B00221A700B4B93F82130AE
S11391AC03F00403002B25D0002363760F4B2022FD
S11391BC1A700F4B984700F034BC00BF080700200E
S11391CCD8060020D40600208E0000209A0000202F
S11391DC9C000020FC060020658A00008000002012
S11391EC090700200A070020CC060020D006002026
S11391FCDD850000A24B93F820301B09DBB29B00E9
S113920CDAB2A04B1A70A04B1A889E4B1B789BB2F7
S113921CD31A9BB2143B9AB29B4B1A80637E03F015
S113922C0F03022B06D1964B93F8213003F03F0326
S113923C122B22D0944B1B88002B06D1904B93F805
S113924C213003F00303002B17D08D4B1A7E237AA5
S113925C9A4240F00D838A4B5A7E637A9A4240F0CC
S113926C0783874B9A7EA37A9A4240F00183844BFE
S113927CDA7EE37A9A4240F0FB82814B93F82130F8
S113928C03F01003002B63D0238A002B60D004F16D
S113929C0C03228A114618467C4B9847784B1A7F4C
S11392AC7B4B1B789A4253D1754B5A7F784B5B7826
S11392BC9A424DD1724B9A7F754B9B789A4247D107
S11392CC6F4BDA7F724BDB789A4241D1704B1B782F
S11392DC23736F4B5B7863736D4B9B78A3736C4BED
S11392ECDB78E373E37E002B2BD1227EA37ED31A8F
S11392FCDBB2FB73FA7BA37DDB08DBB2D31ADBB2E4
S113930CFB73A27DFB7B1344DBB2A37597F90F307F
S113931C002B03DAFB7B5B42DBB2FB73FA7BE37D52
S113932C9B08DBB2D31ADBB2FB73E27DFB7B1344E9
S113933CDBB2E375A37DDB08DAB2E37D1344DBB265
S113934C2376544B01221A70237EA37600232382A6
S113935C637E03F00F03013B072B00F23C8301A255
S113936C52F823F091930000D99300005395000018
S113937CA7970000199800005F9800007B980000E4
S113938C8B970000434B1B7803F00103002B00F078
S113939C2483032363763F4B40221A7000232382D9
S11393AC394B1B88002B0BD03A4B1B7843F0020330
S11393BCDAB2384B1A70344B1B881846364B984724
S11393CC364B00221A80364B984758E1314B1B78A8
S11393DC03F00103002B00F0AC80294B93F82130EF
S11393EC03F03F03122B40F0A480254B93F820305C
S11393FC03F0F003502B7DDD224B00221A7069E040
S113940C204B1B783633274AD25C274B1A70264BD9
S113941C1B78002B6BD0244B1B78012B06D1194BDA
S113942C1B780133DAB2174B1A7053E01E4B1B78BE
S113943C022B3DD1134B1B7837331A4AD35C042BC4
S113944C36D1104B1B783833164AD35C1B021AB234
S113945C0C4B1B7839331349CB5C1BB213431BB233
S113946C9AB2124B1A80114B1B8840F20A62934237
S113947C28BF13469BB26382638AA3823AE000BF7F
S113948C8E00002008070020CC0600206187000015
S113949C04070020D0060020658A0000CE060020B8
S11394ACDD85000080000020090700200A07002049
S11394BC9F4B1B7837339F4AD35C002B19D09C4BA2
S11394CC1B7837339B4AD25C994B1B781344DAB222
S11394DC974B1A70964B1B781A46974B93F820307F
S11394EC1B09DBB2053B9B009A4289DB02E000BFFF
S11394FC00E000BF032363768F4B1B7E23728E4BDD
S113950C5B7E63728C4B9B7EA3728B4BDB7EE37214
S113951C01208A4B98478A4B42221A7000232382DB
S113952C884B00221A80884B00221A80874B98475C
S113953CA5E0834B20221A70844B9847844B1B68FC
S113954C00225A7672E47C4B93F8213003F0010329
S113955C002B30D0637E03F01003002B2BD1238A15
S113956C002B40F03C82774B1B8801339BB218468E
S113957C724B9847724B1B7843F01003DAB2704B62
S113958C1A70704B1B88002B06D06D4B1B7843F064
S113959C0203DAB26A4B1A706C4B9847012323828C
S11395AC082363760023E37600E000BF624B1122AC
S11395BC83F8212060E1604B93F8213003F0200301
S11395CC002B1ED0634B1B685B4A92F826201202B8
S11395DC594991F827100A4313445E4A1360594BB6
S11395EC1A88554B93F826301B0219B2524B93F838
S11395FC27301BB20B431BB29BB2D31A9AB2514BFA
S113960C1A80504B1B88002B10D0637E03F0100380
S113961C002B0BD14A4B1B7843F00203DAB2484BB4
S113962C1A70484B1B881846444B9847424B93F886
S113963C22309BB21B029AB23F4B93F823309BB25D
S113964C13449AB2444B1A80A28A434B1B889A4205
S113965C03D3414B1B88002B02D1A28A3E4B1A80A8
S113966C3D4B1B886382364B1B7803F00303002BA2
S113967C00F0B781344B00221A80344B9847304B9E
S113968C1B7803F02003002B09D02F4B00221A80E7
S113969C00236376284B142283F82120ECE0284B1A
S11396AC1B7803F01003002B0DD0274B00221A80DB
S11396BC01232382042363760023E3761E4B1122B9
S11396CC83F82120D8E0204B1B88002B19D01C4B8D
S11396DC1B7803F00103002B01D000232382238A7F
S11396EC002B0BD1628A184B1B889A4202D2628AD5
S11396FC154B1A80144B1B88238202E0228A124BCE
S113970C1A800023E376154B1B68124A13600E4B28
S113971C1B88002B24D0238A002B21D0238A2833A6
S113972C9AB2084B1A80044B182283F82120A6E025
S113973C08070020800000208E000020658A0000AD
S113974CD0060020CC060020CE060020DD850000CB
S113975CD4060020C40600200A070020C8060020F6
S113976CA24B1B7803F00203002B00F03A81A04BB0
S113977C28221A809F4B102283F821207FE09B4BD8
S113978C1B7803F00103002B6FD000236376974BF7
S113979C10221A70984B984767E0954B1B88002B46
S11397AC04D0934B1B881846944B9847914B93F8D1
S11397BC213003F00103002B17D08C4B1B7803F0E2
S11397CC0103002B06D0072363760023A376002322
S11397DC238201E0062363760120884B9847834B50
S11397EC10221A70844B984742E0804B1B7803F08C
S11397FC0103002B04D0052363760023238210E19C
S113980C7B4B1B88002B00F0EE8031E0784B1B88DF
S113981C002B04D0764B1B881846784B9847754B15
S113982C93F8213003F00103002B0CD0072363764B
S113983C0023A3760120714B98476C4B10221A70AD
S113984C6D4B984714E06A4B1B88002B00F0E880A2
S113985C0EE0664B1B7803F00103002B00F0BB8079
S113986C072363760023A376B5E000BFB3E000BF03
S113987C604B102283F821205D4B28221A805D4B0B
S113988C502283F820205B4B227A1A77594B627A48
S113989C5A77584BA27A9A77564BE27ADA77554B29
S11398AC227B1A76534B627B5A76524BA27B9A7666
S11398BC504BE27BDA764F4B06225A724D4BA28800
S11398CC9A824C4BE288DA824D4B4E4A12881A80AB
S11398DC4D4B4C4A52881A804C4B22881A804C4B64
S11398EC62881A80637E03F01003002B09D0414A6E
S11398FC404B002183F8231093F8233082F8223054
S113990C07E03C4B062283F822203A4B0A2283F8C8
S113991C2320384B40221A72364A354B1B881B0ABB
S113992C9BB2DBB29370334B314A1288D2B2DA70E9
S113993C304A304B002183F8271093F8273082F8F3
S113994C26302C4B00229A842A4C324B98470346DF
S113995CDB439BB2A384274B45221A70254B002270
S113996C5A70244A234B0021D971DB7993712A4B09
S113997C1B8801339AB2284B1A801E4A264B1B882B
S113998C1B0A9BB2DBB213711A4B234A1288D2B254
S113999C5A71184B00225A81164C204B9847034697
S11399ACDB439BB26381114B00221A7040E000BF71
S11399BC37E000BF35E000BF33E000BF31E000BF4B
S11399CC2FE000BF2DE000BF2BE000BF29E000BF5B
S11399DC27E000BF25E000BF23E000BF21E000BF6B
S11399EC1FE000BF1DE000BF1BE000BFD00600203D
S11399FCCC0600208E000020DD850000658A000066
S1139A0C9A0000206C0000209C0000209E00002086
S1139A1CA000002075890000FA060020B58800001B
S1139A2C00BF054B00221A80044B00221A7000BFA1
S1139A3C1437BD4690BD00BFCC060020D0060020D4
S1139A4C80B483B000AF0346FB80FB881B021AB2C0
S1139A5CFB881B0A9BB21BB213431BB29BB2184666
S1139A6C0C37BD4680BC704780B582B000AF1C4B30
S1139A7C1B780133DAB21A4B1A701A4B00221A7083
S1139A8C25E0184B1B781A4613465B0013449B00C5
S1139A9C154A13447B607B681A887B685B88134384
S1139AAC9BB2002B0DD00E4B1B781A467B689B7A0D
S1139ABCD31A772B05DD7B680422002118460B4B47
S1139ACC9847084B1B780133DAB2064B1A70054BD6
S1139ADC1B78072BD5D900BF0837BD4680BD00BF06
S1139AEC72070020700700200C07002059B90000F1
S1139AFC90B583B000AF78603960524B00221A7075
S1139B0C29E0504B1B781A4613465B0013449B0008
S1139B1C4D4A9C182388002B17D06388002B14D033
S1139B2C7B681A8823889A420FD17B6802331A887F
S1139B3C63889A4209D1231D396806221846434B7F
S1139B4C9847434B1B78A37279E03E4B1B78013347
S1139B5CDAB23C4B1A703B4B1B78072BD1D9394BDF
S1139B6C00221A7014E0374B1B781A4613465B001C
S1139B7C13449B00344A9C182388002B02D163881D
S1139B8C002B0AD02F4B1B780133DAB22D4B1A70F1
S1139B9C2C4B1B78072BE6D900E000BF294B1B7814
S1139BAC082B3DD12B4B00221A702B4B00221A7020
S1139BBC244B00221A7022E0224B1B781A461346BF
S1139BCC5B0013449B00204A9C18214B1B781A46BB
S1139BDCA37AD31A1F4A127893420ADD1C4B1A78C3
S1139BECA37AD31ADAB21B4B1A70164B1A781A4B87
S1139BFC1A70144B1B780133DAB2124B1A70114BD6
S1139C0C1B78072BD8D9144B1A780E4B1A700D4BA2
S1139C1C1B781A4613465B0013449B000A4A9C1893
S1139C2C2346042279681846084B9847231D396843
S1139C3C06221846054B9847054B1B78A3720C3724
S1139C4CBD4690BD700700200C0700201DB9000014
S1139C5C72070020730700207107002080B500AF45
S1139C6C384B1B88292B03D8364B00221A8068E00A
S1139C7C344B00221A80344B9B8AB3F5807F03D07B
S1139C8CB3F5007F46D05CE0304B1A88304B1B8810
S1139C9C9A4252D12F4B1A882D4B5B889A424CD145
S1139CAC2D4B2E4A114618462D4B9847264B4FF4F4
S1139CBC00729A822B4B2949062218462A4B984744
S1139CCC264B062229491846274B9847284B06222F
S1139CDC26491846244B9847224B062219461A4803
S1139CEC214B9847184B184A928BDA84164B164A18
S1139CFCD28B1A85144B164A12889A83124B144A27
S1139D0C5288DA83104B4FF4C1629A810D4B2A228C
S1139D1C1A8012E00D4B1A880D4B1B889A420ED1F7
S1139D2C0C4B1A880A4B5B889A4208D10A4B0B4A93
S1139D3C114618460A4B984701E000BF00E000BFEB
S1139D4C00BF80BDCC06002080000020A6000020AF
S1139D5C6C000020A80000209C000020960000202D
S1139D6CFD9A0000A00000201DB90000780000201E
S1139D7C8600002080B582B000AF604B1A88604B1F
S1139D8C1B889A420BD15F4B1A885F4B1B889A42F3
S1139D9C05D106225D495E485E4B98479CE0574BC3
S1139DAC1A885D4B1B8853409AB25C4B1B8813403A
S1139DBC9BB2002B0BD1534B1A88574B5B885340E7
S1139DCC9AB2564B5B8813409BB2002B08D0544B71
S1139DDC1A88544B1A80524B5A88524B5A8007E0BB
S1139DEC464B1A884F4B1A80464B1A884D4B5A8057
S1139DFC4D4B00221A701BE04B4B1B781A46134632
S1139E0C5B0013449B00494A13447B60454B1A88FE
S1139E1C7B681B889A4205D1424B5A887B685B88C5
S1139E2C9A420AD0404B1B780133DAB23E4B1A707B
S1139E3C3D4B1B78072BDFD900E000BF3A4B1B7856
S1139E4C082B42D10622FF213148394B98472D4B20
S1139E5C062200211846364B9847364B06223649C3
S1139E6C18462C4B9847354B062233491846294B38
S1139E7C9847334B2B4A12881A80324B294A528802
S1139E8C1A80314B244A12881A801C4B224A52885D
S1139E9C1A801F4B4FF480729A821D4B4FF48072C0
S1139EACDA811B4B08221A82194B06229A74184B1E
S1139EBC0422DA74164B4FF4C1629A81234B244A60
S1139ECC1A60244B2A221A8015E07B68043306227C
S1139EDC19460F480F4B9847164B0622164918463D
S1139EEC0C4B98470A4B08229A811A4B1B880E3349
S1139EFC9AB2184B1A800837BD4680BD9E000020CC
S1139F0CC4B90000A0000020C6B90000BCB9000010
S1139F1C800000201DB900006C000020740000209B
S1139F2C700000206C070020700700200C07002034
S1139F3C59B900008600002078000020960000200B
S1139F4CA6000020A80000209C000020C4060020CD
S1139F5CB6000020CC06002080B584B000AF786039
S1139F6C39607B680B4A934203D04E210A480B4B51
S1139F7C98473B680A4AA2FB03235B0DFB607B6892
S1139F8C24331A46FB68DBB2136000BF1037BD469E
S1139F9C80BD00BF00800440C8B900007584000077
S1139FAC6BCA5F6B80B584B000AF786039607B6836
S1139FBC264A934203D095212548264B98473B6863
S1139FCC23F4873323F01603002B03D09921204864
S1139FDC204B98477B680C331B68FB60FB6823F0B1
S1139FEC1603FB603B68DBB2FA681343FB607B68C7
S1139FFC0C331A46FB6813607B6808331B68FB60E0
S113A00CFB6823F00E03FB603B681B0ADBB2FA68A7
S113A01C1343FB607B6808331A46FB6813607B6848
S113A02C3C331B68FB60FB6823F00103FB603B685B
S113A03C1B0CDBB2FA681343FB607B683C331A4697
S113A04CFB68136000BF1037BD4680BD0080044020
S113A05CC8B900007584000080B584B000AF786086
S113A06C396007F10803FB607B681E4A934204D0F5
S113A07C4FF481711C481D4B98473B68002B04D14D
S113A08C40F203111848194B98473B681A78FB683F
S113A09C1A70FB6801333A6852781A70FB68023301
S113A0AC3A6892781A70FB6803333A68D2781A705B
S113A0BC7B6814331A46BB6813600023BB603B688F
S113A0CC1A79FB681A70FB6801333A6852791A7072
S113A0DC7B6818331A46BB68136000BF1037BD4643
S113A0EC80BD00BF00800440C8B900007584000026
S113A0FC80B582B000AF78607B68184A934204D074
S113A10C4FF4AC711648174B98477B6808331A46C2
S113A11C7B6808331B6843F0100313607B680833B7
S113A12C1A467B6808331B6843F0010313607B6891
S113A13C0C331A467B680C331B6843F00103136021
S113A14C7B6808331A467B6808331B6843F010039A
S113A15C136000BF0837BD4680BD00BF00800440BB
S113A16CC8B900007584000080B489B000AFF860F1
S113A17CB9607A600023FB61FB6810331B68BB6118
S113A18CBB699BB27B61FB695A1CFA611A46BB68BA
S113A19C1344BA69120CD2B21A70FB695A1CFA61D4
S113A1AC1A46BB681344BA69120ED2B21A707B6990
S113A1BC9A1F7B689342A8BF13463B6109E0FB6975
S113A1CCBA681344FA68103212681A60FB690433D3
S113A1DCFB613B691A1FFB699A42F0DAFA693B6925
S113A1EC9A425EDAFB6810331B68BB613B69DA1E6A
S113A1FCFB699A4220D1FB695A1CFA611A46BB6866
S113A20C1344BA69D2B21A70FB695A1CFA611A4621
S113A21CBB681344BA69120AD2B21A70FB695A1C8D
S113A22CFA611A46BB681344BA69120CD2B21A709A
S113A23CFB690133FB6134E03B699A1EFB699A426A
S113A24C16D1FB695A1CFA611A46BB681344BA69E5
S113A25CD2B21A70FB695A1CFA611A46BB681344D1
S113A26CBA69120AD2B21A70FB690233FB6118E0A4
S113A27C3B695A1EFB699A4213D1FB695A1CFA6159
S113A28C1A46BB681344BA69D2B21A70FB69033319
S113A29CFB6106E0FB6810331B68BB61FB6904338C
S113A2ACFB617B699A1EFB699A42F3DC7B69063B72
S113A2BC7B617A697B689A4202DD7B695B4200E0D0
S113A2CC7B6918462437BD4680BC704780B584B082
S113A2DC00AFF860B9607A60FB68154A934204D009
S113A2EC40F27F211348144B9847BB68002B04D1D0
S113A2FC4FF420710F48104B98477B68002B04DCFB
S113A30C40F281210B480C4B9847FB6834331B6893
S113A31C03F03F03002B01D1002305E07A68B968F0
S113A32CF868064B9847034618461037BD4680BD5F
S113A33C00800440C8B900007584000075A10000B9
S113A34C80B487B000AFF860B9607A6000237B6199
S113A35C7B6840F2FE72934202DD7B685B4296E0BE
S113A36C7B680E3B3B617B695A1C7A611A46BB685D
S113A37C13441B781B041A463B6913433B617B69EA
S113A38C5A1C7A611A46BB6813441B781B061A467E
S113A39C3B6913433B61FB6810331A463B691360FA
S113A3AC0AE0FB68103319467B69BA6813441B68CE
S113A3BC0B607B6904337B617B681A1F7B699A424F
S113A3CCEFDA7A697B689A425BD07B68DA1E7B6928
S113A3DC9A4225D17B695A1C7A611A46BB6813448C
S113A3EC1B783B617B695A1C7A611A46BB6813441F
S113A3FC1B781B021A463B6913433B617B695A1C4D
S113A40C7A611A46BB6813441B781B041A463B69D1
S113A41C13433B61FB6810331A463B69136030E00D
S113A42C7B689A1E7B699A4219D17B695A1C7A61A2
S113A43C1A46BB6813441B783B617B695A1C7A61CE
S113A44C1A46BB6813441B781B021A463B69134318
S113A45C3B61FB6810331A463B69136011E07B685F
S113A46C5A1E7B699A420CD17B695A1C7A611A4632
S113A47CBB6813441B783B61FB6810331A463B6979
S113A48C1360FB6838331A46012313607B68184643
S113A49C1C37BD4680BC704780B584B000AFF860F3
S113A4ACB9607A60FB68154A934204D040F28E314D
S113A4BC1348144B9847BB68002B04D140F28F31DE
S113A4CC0F48104B98477B68002B04DC4FF46471E5
S113A4DC0B480C4B984700BFFB6838331B6803F0E0
S113A4EC0103002BF8D17A68B968F868064B9847D1
S113A4FC034618461037BD4680BD00BF008004409B
S113A50CC8B90000758400004DA3000080B582B06A
S113A51C00AF786039607B680F4A934204D040F2F4
S113A52C35410E480E4B98473B6823F07F03002BB4
S113A53C04D04FF487610948094B98477B6804336E
S113A54C19467B6804331A683B68DB4313400B6081
S113A55C00BF0837BD4680BD00800440C8B9000068
S113A56C7584000080B584B000AF78600B46FB7036
S113A57C7B680C4A934204D04FF48B610A480B4B12
S113A58C98477B681B68FB60FB78002B05D07B68C5
S113A59C04331B68FA681340FB60FB6818461037D9
S113A5ACBD4680BD00800440C8B90000758400001D
S113A5BC80B582B000AF786039607B680C4A9342F6
S113A5CC04D040F28D410B480B4B98473B6823F069
S113A5DC7F03002B04D04FF492610648064B984736
S113A5EC7B683A681A6000BF0837BD4680BD00BF5F
S113A5FC00800440C8B900007584000080B582B0A6
S113A60C00AF78600B46FB707B68144A934204D00D
S113A61C40F2DC411248134B984700BF7B6820334F
S113A62C1B6803F00103002BF8D17B6820331A4616
S113A63CFB78DB00DBB243F00103136000BF7B68E3
S113A64C20331B6803F00103002BF8D17B683033F3
S113A65C1B689BB218460837BD4680BD0080044079
S113A66CC8B900007584000080B582B000AF786072
S113A67C39607B68002B04D140F26B211348144BD6
S113A68C98473B68002B04D14FF41B710F48104BB7
S113A69C9847104B1B6803F0E043002B06D00D4B7E
S113A6AC1A680D4B1340B3F1805F02D14FF0FF33A6
S113A6BC08E00A4B1A687B681A60094B1A683B68F5
S113A6CC1A60002318460837BD4680BD38BA00000E
S113A6DC7584000000E00F400000FF70E0E10F40C3
S113A6ECE4E10F4080B483B000AF78607B68B3F1D1
S113A6FC402F43D07B68264A93423FD07B68254A3F
S113A70C93423BD07B68244A934237D07B68234ADC
S113A71C934233D07B68224A93422FD07B68214AE0
S113A72C93422BD07B68204A934227D07B681F4AE4
S113A73C934223D07B681E4A93421FD07B681D4AE8
S113A74C93421BD07B681C4A934217D07B681B4AEC
S113A75C934213D07B681A4A93420FD07B68194AF0
S113A76C93420BD07B68184A934207D07B68174AF4
S113A77C934203D07B68164A934201D1012300E033
S113A78C0023DBB218460C37BD4680BC704700BFB3
S113A79C00800540005000400090054000600040DF
S113A7AC00A005400070004000B00540004002408D
S113A7BC00C005400050024000D00540006002403B
S113A7CC00E005400070024000F0054000D003405A
S113A7DC0000064080B584B000AFF8600B467A6088
S113A7ECFB72F868244B98470346002B03D1E421F1
S113A7FC2248234B98477B68002B09D07B68012B9C
S113A80C06D07B68022B03D0E6211C481C4B9847CE
S113A81CFB6803F5806319467B6803F00103002B86
S113A82C06D0FB6803F580631A68FB7A134306E0D1
S113A83CFB6803F580631B68FA7AD24313400B6000
S113A84CFB6803F5846319467B6803F00203002B51
S113A85C06D0FB6803F584631A68FB7A134306E09D
S113A86CFB6803F584631B68FA7AD24313400B60CC
S113A87C00BF1037BD4680BDF1A60000A4BA00008D
S113A88C7584000080B584B000AFF8607A603B60DA
S113A89C0B46FB72F868874B98470346002B04D190
S113A8AC4FF4DD718448854B98477B68012B0DD0A0
S113A8BC7B68022B0AD07B68042B07D07B680C2B9B
S113A8CC04D04FF4DF717C487C4B98473B68082BD1
S113A8DC16D03B680A2B13D03B680C2B10D03B686A
S113A8EC092B0DD03B680B2B0AD03B680D2B07D0E2
S113A8FC3B68002B04D040F2C5116F486F4B98474E
S113A90CFB6803F5A06319467B6803F00103002B75
S113A91C06D0FB6803F5A0631A68FB7A134306E0C0
S113A92CFB6803F5A0631B68FA7AD24313400B60EF
S113A93CFB6803F2045319467B6803F00203002BF3
S113A94C06D0FB6803F204531A68FB7A134306E03F
S113A95CFB6803F204531B68FA7AD24313400B606E
S113A96CFB6803F5A16319467B6803F00403002B11
S113A97C06D0FB6803F5A1631A68FB7A134306E05F
S113A98CFB6803F5A1631B68FA7AD24313400B608E
S113A99CFB6803F5A36319467B6803F00803002BDB
S113A9AC06D0FB6803F5A3631A68FB7A134306E02D
S113A9BCFB6803F5A3631B68FA7AD24313400B605C
S113A9CCFB6803F20C5319463B6803F00103002B9C
S113A9DC06D0FB6803F20C531A68FB7A134306E0A7
S113A9ECFB6803F20C531B68FA7AD24313400B60D6
S113A9FCFB6803F5A26319463B6803F00203002BC2
S113AA0C06D0FB6803F5A2631A68FB7A134306E0CD
S113AA1CFB6803F5A2631B68FA7AD24313400B60FC
S113AA2CFB6803F2145319463B6803F00403002B30
S113AA3C06D0FB6803F214531A68FB7A134306E03E
S113AA4CFB6803F214531B68FA7AD24313400B606D
S113AA5CFB6803F21C5319463B6803F00803002BF4
S113AA6C06D0FB6803F21C531A68FB7A134306E006
S113AA7CFB6803F21C531B68FA7AD24313400B6035
S113AA8CFB6803F5A56319463B68002B06D1FB68EC
S113AA9C03F5A5631A68FB7A134306E0FB6803F518
S113AAACA5631B68FA7AD24313400B6000BF1037BE
S113AABCBD4680BDF1A60000A4BA00007584000058
S113AACC80B582B000AF78600B46FB701346BB7048
S113AADC78680B4B98470346002B04D14FF4517103
S113AAEC0848094B9847FB789B001A467B6813442B
S113AAFC1A46BB78136000BF0837BD4680BD00BF43
S113AB0CF1A60000A4BA00007584000090B583B0CF
S113AB1C00AF78600B46FB7078680D4B9847034682
S113AB2C002B04D140F204410A480B4B9847FB78A4
S113AB3C012219467868094B9847F97808230122B1
S113AB4C7868074CA04700BF0C37BD4690BD00BFCA
S113AB5CF1A60000A4BA000075840000E1A700006F
S113AB6C91A8000090B583B000AF78600B46FB70E1
S113AB7C78680D4B98470346002B04D140F21F51C3
S113AB8C0A480B4B9847FB78022219467868094B04
S113AB9C9847F978082301227868074CA04700BF2E
S113ABAC0C37BD4690BD00BFF1A60000A4BA00004E
S113ABBC75840000E1A7000091A8000090B583B053
S113ABCC00AF78600B46FB7078680D4B98470346D2
S113ABDC002B04D140F2C6510A480B4B9847FB7822
S113ABEC022219467868094B9847F97808230422FD
S113ABFC7868074CA04700BF0C37BD4690BD00BF1A
S113AC0CF1A60000A4BA000075840000E1A70000BE
S113AC1C91A8000080B483B000AF78607B685E4A72
S113AC2C934200F0AF807B685C4A934200F0AA80A8
S113AC3C7B685B4A934200F0A5807B68594A934237
S113AC4C00F0A0807B68584A934200F09B807B689C
S113AC5C564A934200F096807B68554A934200F022
S113AC6C91807B68534A934200F08C807B68524AF3
S113AC7C934200F087807B68504A934200F08280B4
S113AC8C7B684F4A93427DD07B684E4A934279D07D
S113AC9C7B684D4A934275D07B684C4A934271D081
S113ACAC7B684B4A93426DD07B684A4A934269D085
S113ACBC7B68494A934265D07B68484A934261D089
S113ACCC7B68474A93425DD07B68402B5AD07B68A3
S113ACDCB3F1102F56D07B68424A934252D07B6812
S113ACEC414A93424ED07B68404A93424AD07B6897
S113ACFC3F4A934246D07B683E4A934242D07B689B
S113AD0CB3F1101F3ED07B683B4A93423AD07B6828
S113AD1C3A4A934236D07B68394A934232D07B68A4
S113AD2C384A93422ED07B68374A93422AD07B68A8
S113AD3C364A934226D07B68354A934222D07B68AC
S113AD4C344A93421ED07B68334A93421AD07B68B0
S113AD5C324A934216D07B68314A934212D07B68B4
S113AD6C304A93420ED07B68B3F1202F0AD07B6813
S113AD7C2D4A934206D07B68082B03D07B682B4A60
S113AD8C934201D1012300E00023DBB218460C37B7
S113AD9CBD4680BC704700BF0100100002001000CB
S113ADAC000110000002100000041000000110103B
S113ADBC000210100004101000401010005010205D
S113ADCC01000020020000200400002008000020E4
S113ADDC10000020200000204000002080000020F3
S113ADEC0001002000400010001010100001102081
S113ADFC8000003010000030000100100002001030
S113AE0C1000001020000010200000300100101071
S113AE1C02001010040010100800101001000010A3
S113AE2C020000100400001001001020001010009B
S113AE3C80B584B000AF78607868224B984703469D
S113AE4C002B04D140F2B9111F48204B98477B6862
S113AE5C1B0F1F4A52F8233018467B681B0F1C4AE1
S113AE6C52F823301A687B6899B27B681B0C03F088
S113AE7C1F0301FA03F3134303600023FB6002E096
S113AE8CFB680133FB60FB680F2BF9D97B681B0F44
S113AE9C0F4A52F8233018467B681B0F0C4A52F8A1
S113AEAC23301A687B6899B27B681B0C03F01F0370
S113AEBC01FA03F3DB431340036000BF1037BD46B4
S113AECC80BD00BF21AC000084BB00007584000071
S113AEDC10BB000080B582B000AF78607868124B6C
S113AEEC98470346002B04D14FF4FC710F48104BC8
S113AEFC98477B681B0F0F4A52F8233018467B681F
S113AF0C1B0F0C4A52F823301A687B6899B27B6881
S113AF1C1B0C03F01F0301FA03F31343036000BF7C
S113AF2C0837BD4680BD00BF21AC000084BB0000C7
S113AF3C758400001CBB000080B400AF014B024AB6
S113AF4C1A60FEE70CED00E00400FA0501387FF40A
S113AF5CFDAF704700BF00BF80B586B000AF78600E
S113AF6C794B1B6803F0E043002B06D0764B1A6830
S113AF7C764B1340B3F1805F03D17B68002BC0F296
S113AF8CDE80734B1B683B61724B1B68FB603B6937
S113AF9C43F400633B613B6923F480033B61FB682E
S113AFAC43F40063FB606A4A3B691360694AFB68BB
S113AFBC13603B6903F00203002B04D07B6803F09D
S113AFCC0203002B09D03B6903F00103002B2BD0A7
S113AFDC7B6803F00103002B26D17B6863F0030329
S113AFEC3A6913403B615A4A3B691360FB68002B76
S113AFFC09DAFB6803F07003302B0CD0FB6803F008
S113B00C7003702B07D0FB68002B09DB3B6903F042
S113B01C3003302B04D14FF480504F4B984703E04E
S113B02C4FF400204C4B98473B6923F45F5323F0B7
S113B03C30033B617A6843F2F07313403A6913436B
S113B04C3B61FA68454B1340FB607A68444B1340F0
S113B05CFA681343FB607B68DB0003F04003FA6877
S113B06C1343FB603F4B40221A60FB68002B06DA4B
S113B07C384AFB681360364A3B69136005E0344A6E
S113B08C3B691360334AFB6813601020324B9847BA
S113B09C3B6923F0F86323F003033B617A68324B7A
S113B0AC13403A6913433B61FB6823F0FC53FB6088
S113B0BC7B6803F0FC53FA681343FB607B6803F072
S113B0CC8043002B0ED03B6943F480033B61FB6847
S113B0DC23F48003FB607A68244B1340FA6813430F
S113B0ECFB6003E0FB6823F08043FB607B6803F4A4
S113B0FC0063002B19D14FF400437B6108E01C4B17
S113B10C1B6803F04003002B06D17B69013B7B6178
S113B11C7B69002BF3D100E000BF3B6923F400638F
S113B12C3B61FB6823F40063FB60094A3B691360D1
S113B13C084AFB6813601020074B984700E000BFD7
S113B14C1837BD4680BD00BF00E00F400000FF7003
S113B15C60E00F4070E00F4059AF00008FDFFF7FBD
S113B16C3020008058E00F400300C007000040402E
S113B17C50E00F4080B485B000AF944B1B68FB606B
S113B18C934B1B687B607B68002B03DA7B6803F0B2
S113B19C700302E0FB6803F03003202B45D0202B16
S113B1AC04D8002B09D0102B10D079E0602B6FD071
S113B1BC702B71D0302B67D072E0FB689B0903F0C5
S113B1CC1F03844A52F82330BB606BE0824B1B682C
S113B1DC03F0E043002B06D07F4B1A687F4B1340DF
S113B1ECB3F1805F02D17E4BBB601DE07A4B1A68D1
S113B1FC7A4B13407B4A934204D1774B1B689BB226
S113B20C022B0BD0744B1A68744B1340764A93423E
S113B21C07D1714B1B689BB2002B02D1734BBB60E3
S113B22C02E0734BBB603DE03CE06B4B1B6803F0EE
S113B23CE043002B06D0684B1A68684B1340B3F1FB
S113B24C805F02D16B4BBB601DE0634B1A68634B90
S113B25C1340644A934204D15F4B1B689BB2022B8C
S113B26C0BD05D4B1A685D4B13405F4A934207D178
S113B27C594B1B689BB2002B02D15F4BBB6002E0A5
S113B28C5E4BBB600EE00DE047F23053BB6009E04F
S113B29C4FF48003BB6005E04FF40043BB6001E056
S113B2AC00238EE07B68002B04DA7B6803F40063D4
S113B2BC002B07D07B68002B47DBFB6803F400638F
S113B2CC002B42D14E4B1B683B60434B1B6803F075
S113B2DCE043002B06D0404B1A68404B1340B3F1AB
S113B2EC805F0FD13B685B09C3F308030233BA6870
S113B2FC02FB03F23B6803F01F030233B2FBF3F3CC
S113B30CBB600EE03B685B09C3F30803BA6802FB3D
S113B31C03F23B6803F01F0301335B00B2FBF3F34E
S113B32CBB603B6803F48043002B02D0BB685B0812
S113B33CBB603B6803F40043002B02D0BB689B0842
S113B34CBB60FB6843F48003FB60FB6803F480037D
S113B35C002B35D07B68002B29DA7B6803F0804303
S113B36C002B1AD07B68002B04DA7B6803F400638F
S113B37C002B07D07B68002B0FDBFB6803F4006306
S113B38C002B0AD1BB685A007B689B0D03F07F032A
S113B39C0133B2FBF3F3BB6012E07B68DB0D03F00B
S113B3AC3F030133BA68B2FBF3F3BB6008E0FB68FC
S113B3BCDB0D03F00F030133BA68B2FBF3F3BB608C
S113B3CCBB6818461437BD4680BC704760E00F401C
S113B3DC70E00F4028BB000000E00F400000FF703D
S113B3ECC0E1E4000000011000000310001BB700D2
S113B3FC0024F40070383900C0C62D0000093D004B
S113B40C64E00F4080B400AF044A044B1B6843F063
S113B41C0503136000BFBD4680BC704710E000E01C
S113B42C80B400AF044A044B1B6843F0020313605E
S113B43C00BFBD4680BC704710E000E080B582B010
S113B44C00AF78607B68002B03D07B68B3F1807FFE
S113B45C03D9D0210548064B9847064A7B68013B23
S113B46C136000BF0837BD4680BD00BFF0BB0000B1
S113B47C7584000014E000E080B483B000AF786001
S113B48C7B680A4A934207D07B68094A934203D0EB
S113B49C7B68084A934201D1012300E00023DBB20C
S113B4AC18460C37BD4680BC704700BF00C0004036
S113B4BC00D0004000E0004080B586B000AFF860DA
S113B4CCB9607A603B60F868444B98470346002B9C
S113B4DC04D140F20D114248424B98477B68002B33
S113B4EC04D14FF487713E483E4B98473E4B1B6842
S113B4FC03F0E043002B1ED03B4B1A683B4B13402C
S113B50CB3F1805F17D0384B1A68384B1340384A64
S113B51C934204D1344B1B689BB2022B0BD0324B9D
S113B52C1A68324B1340334A934206D12E4B1B6894
S113B53C9BB2002B01D1102300E008237A6802FB94
S113B54C03F2BB689A4204D940F20F112448254BEC
S113B55C9847F868284B98477B681A01BB689A424D
S113B56C0CD9FB6830331A46FB6830331B6843F044
S113B57C200313607B685B087B6008E0FB68303356
S113B58C1A46FB6830331B6823F020031360BB6836
S113B59CDA007B68B2FBF3F301335B087B61FB6875
S113B5AC24331A467B699B091360FB6828331A46BB
S113B5BC7B6903F03F031360FB682C331A463B682A
S113B5CC1360FB6818331A4600231360F8680B4B9E
S113B5DC984700BF1837BD4680BD00BF85B4000036
S113B5EC5CBC00007584000000E00F400000FF709C
S113B5FC000001100000031069B600000DB6000035
S113B60C80B582B000AF78607868114B98470346D8
S113B61C002B04D14FF4CF710E480F4B98477B6825
S113B62C2C331A467B682C331B6843F010031360CD
S113B63C7B6830331A467B6830331B6843F44073A1
S113B64C43F00103136000BF0837BD4680BD00BF43
S113B65C85B400005CBC00007584000080B582B029
S113B66C00AF78607868154B98470346002B04D1DB
S113B67C4FF4DF711248134B984700BF7B681833A3
S113B68C1B6803F00803002BF8D17B682C331A4693
S113B69C7B682C331B6823F0100313607B683033F6
S113B6AC1A467B6830331B6823F4407323F0010380
S113B6BC136000BF0837BD4680BD00BF85B40000D1
S113B6CC5CBC00007584000080B582B000AF78606B
S113B6DC78680D4B98470346002B04D140F209417E
S113B6EC0A480B4B98477B6818331B6803F010030C
S113B6FC002B02D17B681B6801E04FF0FF33184626
S113B70C0837BD4680BD00BF85B400005CBC00009A
S113B71C7584000080B500AF0348044B9847024879
S113B72C034B984700BF80BD00501020E1AE0000D1
S113B73C3DAE000080B586B000AF4648464B9847F6
S113B74C0C214648464B98477F214648464B984720
S113B75C00214448454B9847786179694148444BEA
S113B76C9847444B9847034619463E48424B9847E2
S113B77C16213C48414B98473A48414B9847012184
S113B78C3848404B984778613F4B9847034603F53C
S113B79C9C5308333B610AE001213248394B9847EA
S113B7AC7861394B984702463B699A4205D27B69CA
S113B7BC03F00403002BEFD000E000BF08233B721E
S113B7CC00237B722723BB726923FB725B233B73BD
S113B7DC45237B733A463B1D114618462B4B984721
S113B7EC7B68B3F1FF3F19D03B68B3F1FF3F15D031
S113B7FC7B68DBB23B727B681B0ADBB27B727B68B7
S113B80C1B0CDBB2BB723B68DBB2FB723B681B0AE2
S113B81CDBB23B733B681B0CDBB27B7307F1080395
S113B82C194610481A4B98473A7A1A4B1A707A7A76
S113B83C184B5A70BA7A174B9A70FA7A154BDA700D
S113B84C3A7B144B1A717A7B124B5A7100BF18371E
S113B85CBD4680BD20000020E1AE00000050024037
S113B86CC9AB00000080044019A5000071A50000BC
S113B87CBDA5000081B10000659F0000B19F0000D0
S113B88CFDA0000009A60000FD84000075A60000C0
S113B89C65A000007800002080B582B000AF0021C4
S113B8AC0C480D4B9847786079680A480B4B9847BD
S113B8BC7B6803F00103002B07D040F24262084975
S113B8CC0448084B9847034600E000231846083701
S113B8DCBD4680BD0080044071A50000BDA50000DC
S113B8EC80000020D9A2000080B500AF044B1B8857
S113B8FC1A4604490448054B984700BF80BD00BF55
S113B90CCC0600208000002000800440A5A4000088
S113B91C844640EA010313F0030F0DD1242A0BD300
S113B92C2DE9F00FB1E8F80FA0E8F80FA2F124020A
S113B93C242AF7D2BDE8F00F002A05D011F8013BF8
S113B94C00F8013B013AF9D1604670478446002A5D
S113B95C2AD010F0030F04D000F8011B013A23D0B5
S113B96CF7E7282A1CD3A2F128022DE9F00F01F0E5
S113B97CFF0141EA012141EA014141EA01610B461F
S113B98C0C460D460E460F46884689468A468B461B
S113B99CA0E8FA0F283AFBD2BDE8F00F283203D006
S10FB9AC00F8011B013AFBD16046704713
S113B9B800000000FFFFFFFFFFFF0000FFFFFFFF85
S113B9C8433A2F576F726B2F736F66747761726582
S113B9D82F4F70656E424C542F5461726765742FF3
S113B9E844656D6F2F41524D434D335F4C4D335376
S113B9F85F454B5F4C4D3353363936355F43726F71
S113BA087373776F726B732F50726F672F696465E6
S113BA182F2E2E2F6C69622F6472697665726C6999
S113BA28622F65746865726E65742E630000000089
S113BA38433A2F576F726B2F736F66747761726511
S113BA482F4F70656E424C542F5461726765742F82
S113BA5844656D6F2F41524D434D335F4C4D335305
S113BA685F454B5F4C4D3353363936355F43726F00
S113BA787373776F726B732F50726F672F69646576
S113BA882F2E2E2F6C69622F6472697665726C6929
S113BA98622F666C6173682E63000000433A2F5767
S113BAA86F726B2F736F6674776172652F4F706551
S113BAB86E424C542F5461726765742F44656D6FE0
S113BAC82F41524D434D335F4C4D33535F454B5FCC
S113BAD84C4D3353363936355F43726F7373776F12
S113BAE8726B732F50726F672F6964652F2E2E2F18
S113BAF86C69622F6472697665726C69622F67700B
S113BB08696F2E630000000040E00F4044E00F40DE
S113BB1848E00F4000E10F4004E10F4008E10F4006
S113BB2840420F0000201C0080841E000080250075
S113BB38999E36000040380000093D0000803E0010
S113BB4800004B00404B4C0000204E00808D5B00F1
S113BB5800C05D000080700000127A0000007D00C3
S113BB6880969800001BB7000080BB00C0E8CE0098
S113BB78647ADA000024F4000000FA00433A2F57EC
S113BB886F726B2F736F6674776172652F4F706570
S113BB986E424C542F5461726765742F44656D6FFF
S113BBA82F41524D434D335F4C4D33535F454B5FEB
S113BBB84C4D3353363936355F43726F7373776F31
S113BBC8726B732F50726F672F6964652F2E2E2F37
S113BBD86C69622F6472697665726C69622F737915
S113BBE87363746C2E630000433A2F576F726B2F84
S113BBF8736F6674776172652F4F70656E424C542B
S113BC082F5461726765742F44656D6F2F41524DCF
S113BC18434D335F4C4D33535F454B5F4C4D33536A
S113BC28363936355F43726F7373776F726B732F60
S113BC3850726F672F6964652F2E2E2F6C69622FDF
S113BC486472697665726C69622F73797374696357
S113BC586B2E6300433A2F576F726B2F736F6674A2
S113BC68776172652F4F70656E424C542F54617220
S113BC786765742F44656D6F2F41524D434D335F93
S113BC884C4D33535F454B5F4C4D33533639363542
S113BC985F43726F7373776F726B732F50726F6732
S113BCA82F6964652F2E2E2F6C69622F6472697652
S110BCB865726C69622F756172742E6300F1
S903819BE0
